:100000001D28FF3FFF3FFF3F9500030896000B119F
:10001000AB0B1828121D182812112C08F039AA0051
:1000200003102C0D0F39031901302A04AC0086008F
:1000300016088300950E150E090009308500E03082
:100040008600163065009030660009308500E0308B
:100050008600AC009401920164000F3062002030F1
:100060008B00980197011B2164000F306200051A74
:100070002A2905193E28851840283428851834284F
:1000800092132E30840033231308A000130880003D
:10009000840AF33013020319ED29563013070318AD
:1000A000EC287F30130703185928EF301307031883
:1000B000EC2833231308A10013088000840A0630BB
:1000C0001302031DEC281B2118089A001708990039
:1000D0000130A6009212332313088000840A13080B
:1000E000A200332303308E00332313088000840AD8
:1000F0001308A5008E0B74281D30250203198428CF
:100100000F302502031D87280330A6009216A20394
:1001100022088E00332313088000840A8E0B8A285D
:100120005630A1001823921FF82092171B21121796
:100130000408A7002E308400000893000322840ADC
:1001400027080402031D9C2813218B170930A100E6
:10015000182323232923292329231D08A200292327
:100160001D08A30022088E0023088F008F0A292370
:100170008E0BB7288F0BB728292329235630A100CF
:100180001823A60BAA28921ADC282E3084003323C9
:100190001308A00013088000840A33231308A10069
:1001A00013088000840A92301302031D6828332349
:1001B00033235630A100182393010322121BE32896
:1001C00093010322DE280617132101231B211A089D
:1001D00098001908970034281A0898001908970001
:1001E0001321E0308600061486140608AC002A2885
:1001F000D230A7001321051A0D2964000F306200C8
:100200000723A70BFB281B21051A0D2964000F30BB
:1002100062000723A70B0429F8280D230D23051ED0
:10022000F8281B2108008B138B1B13292C08F0398D
:10023000AC008600080017080339A900A90AA80124
:100240000314A80DA90B21292C08F03928048600D5
:10025000AC000800E13090000D230D23051E34286A
:100260000D23900A03194129051A30291708FC3972
:100270009800970A033097051808970498011B21E6
:1002800034281B216400051A42290F306200180827
:100290009A001708990012175C221408A0005C222B
:1002A0001408A1008B170130A600921220089400B8
:1002B00058232108940058232E231E08A2009401DD
:1002C000582303308E002E231E08A5008E0B6329B1
:1002D0001D302502031970290F302502031D7329D3
:1002E0000330A6009216A20322088E002E238E0B46
:1002F0007629232393298E018F01051D9329851CBF
:10030000932964000F3062008E0B7D29051D93290F
:10031000851C932964000F3062008E0B86297B298F
:1003200064000F306200332333231308A10033230A
:10033000332336302102031DAE2933233323130820
:10034000A1003323013021020319DE2902302102EA
:10035000031DDE295630A1001823DE295630A100E6
:1003600018232E232E232E231E08A2002E231E0820
:10037000A30022088E0023088F008F0A2E238E0BE5
:10038000BE298F0BBE292E232E232323A60BB12992
:10039000921AD2295C229408031D4D299230A100A3
:1003A000182323235C22121FD22906171A0898004B
:1003B00019089700132101231B2134285C22121FE6
:1003C000DE291A089800190897001321E0308600EA
:1003D000861406150608AC002A2813218B17180866
:1003E0009A00170899001217332313088F0058300A
:1003F000940058237F308E002E238E0BFC298F0B08
:10040000FA290617D22964000F306200121B2D2A28
:100410001308A406DC229F0B2C2A01232408930036
:10042000DC229301DC225C301402031D502A93016C
:10043000DC225D301402031D502A9301DC22473078
:100440001402031D502A012306170D23061301234E
:10045000980A0319970A1217080013089D008130A3
:100460009300DC2257309300DC229301DC225A30C7
:100470001402031D502A9301DC225D301402031D77
:10048000502A17089300DC2218089300DC22180871
:100490001706A40080309F0012131D089300032A42
:1004A00085108511061701231321E03086000930DD
:1004B0008500861486152A2864000F3062000830F3
:1004C000AD00121B8D2A9301DC221408A4069F0B99
:1004D000832A14089E009301DC2224081402031DC1
:1004E000CD2A12169301DC2247301402031DCD2AB7
:1004F00006170D230D230D230D23980A0319970AC0
:1005000012171E089400080006170D230D230D2353
:100510000D230D23AD0B8D2ACD2A061301231216B0
:1005200081309300DC22121652309300DC229301BA
:10053000DC225A301402031D842A9301DC225D3030
:100540001402031DCD2A17089300DC22180893001B
:10055000DC229301DC225C301402031DCD2A9301BE
:10056000DC229408031DB62A9301DC2294080319A7
:10057000CD2A9301DC2217081402031DCD2A930112
:10058000DC2218081402031DCD2A18081706A4003F
:1005900080309F00121301235C2A851085110617F5
:1005A0000123132109308500E0308600061406156A
:1005B0006530940058232A288B138B1BDC2A940166
:1005C0000830910005100310930C031C86120318C9
:1005D0008616EA2AEB2AEC2AED2AEE2AEF2A0514DF
:1005E0000310061E0310061A0314940CF72AF82AA7
:1005F000F92AFA2AFB2AFC2A910BE22A861605140C
:100600008B1710308C0000008C0B032B0800DC30A3
:100610008C0000008C0B092B080014308D008C011D
:1006200064008C0B102B8D0B0F2B0F306200080019
:10063000200894005823210894005823940158233B
:1006400094015823080004308C0033238C0B252B95
:100650000800332313089D00032208005C221408BD
:100660009E00582308009301083091008518462BFE
:10067000051D362B85110310930C851C3D2B85150C
:10068000051D402B910B362B121508000519362B32
:1006900085101430650085100314930C051D4E2B36
:1006A00016306500851C522B910B362B1215080055
:1006B00008309100163065008515851C5A2B051DE4
:1006C0005A2B0310940C0318772B851014306500F7
:1006D00085108518692B05196B2B16306500851C54
:1006E0006F2B051D712B910B612B121508008511C5
:1006F0000519782B85187A2B8515051D7D2B851CF2
:100700007F2B910B612B1215080052337516513255
:100710003433433DA43DA43DA43D17322309441086
:100720002539433605120932243003322910143298
:1007300046323712863121242D349304D4200932D5
:10074000922094302D0309094732713263353827DE
:100750003229033220200923D204200DC0020C0CC0
:10076000C00C3C303204783289373020C93432042E
:10077000C20C23033A202A23AA0203042A2D323F63
:10078000F21232324332FF2132212133133234212B
:1007900031251632893D89139D3889302403580448
:1007A000950405394928503CC908D803430348300B
:1007B00085048503890C5408580C5039903543251D
:1007C0008C25280373080829C909830913201C02F2
:1007D00002381110100090129332130239200323B3
:1007E00023010312293012303930910201099D0290
:1007F000231B2B01B432900C900DBB0ABA01300BB5
:084000007F007F007F007F00BC
:02400E00F53F7C
:00000001FF
